:020000040000FA
:1000000020308316900083120730990001309F0042
:1000100083160030990051309F000930850083120B
:10002000FF3085001430851DFA30A300A401A5011E
:10003000FA30CD20FA30CD200430B0000330B100CA
:100040000330B2000330B3000730B4000430B50011
:100050000330B6000630B700FF30B8000430C000EF
:100060000330C1000330C2000330C3000530C400B8
:100070000330C5000630C6000630C700FF30C80098
:100080006430CD20363085049F14000000009F1896
:10009000452861301E02031C522805118510A40A50
:1000A000A5017128A40160301E02031C60280511FF
:1000B0008510C830CD200515C830CD200511712818
:1000C0005E301E0203186628A50A7128A5015F305C
:1000D0001E02031870288510C830CD2085147128A1
:1000E00085102408230203187A2805123030832053
:1000F000A401822825082302031882280512403013
:100100008320A50140288400A220AB20851200088E
:10011000A000FF3A031D8E2885160800B820BE20D7
:10012000A00B8E28C420840A872885160330A100DE
:10013000A10B98280000000085120230A100A10B3D
:100140009F2808003F30A2009520A20BA4289520EC
:10015000A20BA7280800F830A200AE28AF28B028CC
:10016000B128B228B328B428B528A20BAD280800BE
:100170001530A2009520A20BBA280800B330A200C7
:100180000000A20BC0280800B430A200000000004C
:1001900000000000A20BC6280800A1006E30A000DD
:1001A000000000000000000000000000A00BD028AC
:1001B000A10BCE2808002A0045006D0069006C00E4
:1001C00069006F002A002800310037002D00300040
:1001D00036002D0030003700290000340034FF3F86
:1001E000FF3FFF3FFF3FFF3FFF3FFF3FFF3FFF3F1F
:1001F000FF3FFF3FFF3FFF3FFF3FFF3FFF3FFF3F0F
:10020000FF3FFF3FFF3FFF3FFF3FFF3FFF3FFF3FFE
:10021000FF3FFF3FFF3FFF3FFF3FFF3FFF3FFF3FEE
:02400E00843FED
:08400000FF3FFF3FFF3FFF3FC0
:0207FE000034C5
:00000001FF
